:0200000480007A
:100000006F00C004732F2034930F8000630AFF0336
:10001000930F90006306FF03930FB0006302FF038A
:10002000170F0080130F0FFE63040F0067000F000F
:10003000732F203463540F006F004000136E9E53E3
:10004000171F00002320CFFD6FF09FFF732540F1A5
:100050006310050073251030635805000F00F00F82
:10006000130E100073000000130E00009702000032
:10007000938282F973905230735020307350303035
:1000800073504030970200809382C2F7638C020065
:10009000739052109302B01A739022307323203061
:1000A000E39E62F873500030970200009382420191
:1000B00073901234732540F173002030B70001FFB4
:1000C000938000F037110F0F1301F1F0B3F120000E
:1000D000B71E000F938E0EF0130E2000639CD149C3
:1000E000B710F00F938000FF37F1F0F01301010F0C
:1000F000B3F12000B70EF000938E0E0F130E3000F8
:10010000639AD147B700FF009380F00F37110F0FAC
:100110001301F1F0B3F12000B70E0F00938EFE0033
:10012000130E40006398D145B7F00FF09380F000B4
:1001300037F1F0F01301010FB3F12000B7FE00F02A
:10014000130E50006398D143B70001FF938000F075
:1001500037110F0F1301F1F0B3F02000B71E000F9D
:10016000938E0EF0130E60006396D041B710F00F1F
:10017000938000FF37F1F0F01301010F33F12000FD
:10018000B70EF000938E0E0F130E70006314D13F64
:10019000B70001FF938000F0B3F01000B70E01FF2D
:1001A000938E0EF0130E80006396D03D1302000074
:1001B000B70001FF938000F037110F0F1301F1F02A
:1001C000B3F12000138301001302120093022000F8
:1001D000E31052FEB71E000F938E0EF0130E900028
:1001E000631AD33913020000B710F00F938000FF99
:1001F00037F1F0F01301010FB3F1200013000000FC
:10020000138301001302120093022000E31E52FC2C
:10021000B70EF000938E0E0F130EA000631CD335A3
:1002200013020000B700FF009380F00F37110F0F8B
:100230001301F1F0B3F120001300000013000000DF
:10024000138301001302120093022000E31C52FCEE
:10025000B70E0F00938EFE00130EB000631CD33157
:1002600013020000B70001FF938000F037110F0F59
:100270001301F1F0B3F120001302120093022000E9
:10028000E31252FEB71E000F938E0EF0130EC00045
:100290006392D12F13020000B710F00F938000FF7C
:1002A00037F1F0F01301010F13000000B3F120004B
:1002B0001302120093022000E31052FEB70EF0006A
:1002C000938E0E0F130ED0006396D12B13020000F5
:1002D000B700FF009380F00F37110F0F1301F1F0FB
:1002E0001300000013000000B3F1200013021200FD
:1002F00093022000E31E52FCB70E0F00938EFE0007
:10030000130EE0006398D12713020000B70001FF2D
:10031000938000F01300000037110F0F1301F1F06C
:10032000B3F120001302120093022000E31052FEEA
:10033000B71E000F938E0EF0130EF000639CD123B6
:1003400013020000B710F00F938000FF13000000AD
:1003500037F1F0F01301010F13000000B3F120009A
:100360001302120093022000E31E52FCB70EF000AD
:10037000938E0E0F130E0001639ED11F1302000017
:10038000B700FF009380F00F13000000130000007F
:1003900037110F0F1301F1F0B3F120001302120017
:1003A00093022000E31E52FCB70E0F00938EFE0056
:1003B000130E10016390D11D1302000037110F0FAF
:1003C0001301F1F0B70001FF938000F0B3F12000BA
:1003D0001302120093022000E31252FEB71E000F18
:1003E000938E0EF0130E20016396D11913020000B4
:1003F00037F1F0F01301010FB710F00F938000FFF9
:1004000013000000B3F12000130212009302200039
:10041000E31052FEB70EF000938E0E0F130E300154
:10042000639AD1151302000037110F0F1301F1F079
:10043000B700FF009380F00F1300000013000000CE
:10044000B3F120001302120093022000E31E52FCBD
:10045000B70E0F00938EFE00130E4001639CD11166
:100460001302000037110F0F1301F1F01300000009
:10047000B70001FF938000F0B3F1200013021200D7
:1004800093022000E31052FEB71E000F938E0EF071
:10049000130E50016390D10F1302000037F1F0F0FA
:1004A0001301010F13000000B710F00F938000FF3D
:1004B00013000000B3F12000130212009302200089
:1004C000E31E52FCB70EF000938E0E0F130E600168
:1004D0006392D10B1302000037110F0F1301F1F0DB
:1004E0001300000013000000B700FF009380F00F1E
:1004F000B3F120001302120093022000E31E52FC0D
:10050000B70E0F00938EFE00130E70016394D10797
:10051000B70001FF938000F033711000930E0000CC
:10052000130E80016318D105B700FF009380F00F10
:1005300033F10000930E0000130E9001631CD103F1
:10054000B3700000930E0000130EA0016394D0035B
:10055000B71011119380101137212222130121228B
:1005600033F02000930E0000130EB0016314D0018D
:10057000631CC0010F00F00F63000E00131E1E006D
:10058000136E1E00730000000F00F00F130E10001A
:1005900073000000731000C00000000000000000A5
:1005A000000000000000000000000000000000004B
:1005B000000000000000000000000000000000003B
:0405C0000000000037
:1010000000000000000000000000000000000000E0
:1010100000000000000000000000000000000000D0
:1010200000000000000000000000000000000000C0
:1010300000000000000000000000000000000000B0
:081040000000000000000000A8
:040000058000200057
:00000001FF
